:020000040800F2
:1000000090190020A901000885150008810C00083E
:1000100000000000000000000000000000000000E0
:10002000000000000000000000000000CD1B0008E0
:10003000000000000000000087150008D11C000827
:10004000BB010008BB010008BB010008BB010008A0
:10005000BB010008BB010008BB010008BB01000890
:1000600000000000BB010008BB010008BB01000844
:10007000BB010008BB010008BB0100080000000034
:10008000BB010008BB01000800000000D51D0008EE
:10009000091E000899200008CD200008BB010008B7
:1000A000BB010008BB010008BB01000809210008D2
:1000B000992100080000000000000000000000007E
:1000C000BB01000800000000BB01000800F002F8BE
:1000D00000F03EF80CA030C8083824182D18671E10
:1000E000A246AB4654465D46AC4201D100F030F822
:1000F0007E460F3EB6460FCC0126334200D0FB1A97
:100100003343A246AB461847B0470000D047000033
:10011000103A02D378C878C1FAD8520701D330C850
:1001200030C101D504680C60704700000023002432
:1001300000250026103A01D378C1FBD8520700D31E
:1001400030C100D50B6070471FB51FBD10B510BD85
:1001500000F090FB1146FFF7F7FF03F021F800F0E5
:10016000A8FB03B4FFF7F2FF03BC00F007FC00009C
:1001700070B505460C46164602E00FCC0FC5103E82
:10018000102EFAD2082E02D303CC03C5083E042E4B
:1001900007D301CC01C5361F03E021782970641C08
:1001A0006D1C761EF9D270BD07488047074800478E
:1001B000FEE7FEE7FEE7FEE7FEE7FEE70448054947
:1001C000054A064B70470000E51C0008CD000008FA
:1001D000901100209019002090150020901500200B
:1001E000F8B5042A2CD3830712D00B78491C03706E
:1001F000401C521E83070BD00B78491C0370401C17
:10020000521E830704D00B78491C0370401C521EF9
:100210008B079B0F05D0C91ADF002023DE1B08C9FE
:100220000AE0FFF7A5FFF8BD1D4608C9FD401C46C2
:10023000B4402C4310C0121F042AF5D2F308C91A87
:10024000521EF0D40B78491C0370401C521EEAD495
:100250000B78491C0370401C012AE4D40978017012
:10026000F8BD7047704770470246C80FC00781430A
:100270004B0030B54B405B009B0D20D01923DB06B3
:10028000C91801231B05994220DB0324A407042578
:100290001346AB400BD3002B04D1EB0613409B005D
:1002A000E34204D401246407002312195941FF23B7
:1002B0001B0599420BD2C9000143500F09E0CB0244
:1002C00004D501430803024305D0054830BDFF2192
:1002D000C905084330BD084607210905884330BDDC
:1002E0000000C07FF0B58B4C0F09254689B0BD4397
:1002F0007BD01D092646AE43FAD00E465E4027400D
:10030000F60F3E43254071D024012142FBD0FF244B
:10031000AD19A4042D1B039501252D05DB02DB0A75
:10032000C9022B43C90A29431E010901040F130FF7
:10033000050121431701880B820391432D098C4647
:10034000A90B1E438A039543B30B9A0396433F09B7
:10035000BA0B9403A74302962E467E430497B646F3
:100360004E19D7190C460196544305977E43371B07
:100370007646BF1B3601B646BE0B3619009676464A
:10038000BC043719009C01D3641C00946400002F46
:1003900001D001263443029E049F754366467E4386
:1003A0000496760034196E0034190094029C019E64
:1003B0001C196643751BAE46069465464519059C97
:1003C00005956C43594375460891691A0191049E3D
:1003D00001465143A41B0491611A009C0791E10658
:1003E00005D061090122114302E072E06EE061096B
:1003F000089D00272C0A2D066918049D7C412A0AB5
:100400002D066918019D6241AC0DAD026D18544175
:10041000079A910D920255196141029A6446584318
:100420005443069B059A5A43121A131B9A0E9B01BA
:100430005B187A41010B0005C3185141220A2006BE
:1004400044195A419A4200D2491C0120400281427B
:1004500003D315230226F64302E014230326F643B2
:100460002020C51AA9401746AF40DA400A4320466B
:100470000399D8400914731819055118039A384381
:10048000D2075140AC4009D00122944006D300224B
:10049000401C5141002C01D1400840001E4A9342AB
:1004A00012D3012203989206904207DB05204007F1
:1004B00009181A480143C012414004E003204007D4
:1004C0000818C10FC907002009B0F0BD0020F107CE
:1004D000FAE705180C464C4111486D42A04115D36E
:1004E00094181A465A410E48644290410ED3012096
:1004F0004A004005824209D35A00824206D359403D
:10050000C90F084AC90700201143DDE7002006494A
:10051000DAE700000000FF07FE070000FFFFFF7F93
:100520000000E0FF0000F07F0000F87F0121C90516
:100530000123411842001B06D3185B0E0AD0C110DC
:100540000722D206891840075242D14201D55200F3
:1005500089187047090208D50146002A03D0C10F47
:10056000C9070020704710467047420202D00020A1
:1005700002497047072109050143F4E70000F87FAD
:10058000F0B5FF252D04C609C209FF2704462E40F9
:100590000137CB093E4348402A402B400746002AFA
:1005A0006BD0002B69D0AA4267D0AB4265D000283F
:1005B00000DA32460125ED0529432C4309022002C9
:1005C000090AD21A4B0C7F24E31A434C000A7C44DC
:1005D000E35C7D242404121914145B00A2188842E1
:1005E00001D3521C00E0400049420C465C432411F8
:1005F0005C43DB016415E318040A5C43C502200D6B
:100600000C4644436419250A5D432303EC0C0D4654
:10061000654300030019EB184C42A34201D35B1859
:10062000401CD4052018002B07D05B00C91804D348
:10063000401C002901D1400840003F2189048A4222
:1006400009D3002A08DC1106090F04D00321490749
:100650004018C00FC007F0BD0122410012068918E2
:100660007F2252069142F6D205214907C84201D5A0
:100670009010F0BDFF20C005F0BD002F00DA32461B
:100680001648AA4207D2AB4205D21902090E17D06A
:10069000F80FC007F0BDFF2563002D06AB42F9D867
:1006A0004900A942F6D8AB4201D1A942F2D0A942F1
:1006B00001D1002101E061004908D0050843F0BDE7
:1006C0001102090EFBD0FF200243D005F0BD0A46FF
:1006D0000146104654E70000BE3F00000000C07F06
:1006E0000102C21504D00123DB071943002A0ADBEB
:1006F0009E239A1A02D40846D0407047FF22410038
:100700001206914201D900207047C017C0437047BC
:100710001F22030C02D10F2200041CD0030E01D1B2
:100720000002083A030F01D10001121F830F01D10B
:100730008000921E002801DB4000521ED205511895
:10074000021251181922904004D3491C002801D1EB
:100750004908490008467047C10FC90700D0404208
:10076000012292071143D3E701218907D0E7000056
:10077000F8B5264C4E00069DA6420AD8A64201D1E5
:10078000002806D15E00A64203D8A6420AD1002A5C
:1007900008D00D242404254233D02946002000F03F
:1007A00090F8F8BD0C461C4311D4994207D0C81AE2
:1007B00002D3EFF30080F8BDEFF30080F8BD801A9C
:1007C00002D3EFF30080F8BDEFF30080F8BD0924F9
:1007D0002407E5008B4207D0581A02D3EFF30080BC
:1007E00006E0EFF3008007E0101A03D3EFF3008078
:1007F000A04303E0EFF30080A043284380F3008888
:10080000F8BD009500F074F8F8BD00000000E0FFAE
:1008100010B5FF231B0644009C421DD84C009C428F
:100820001AD80346124A0B4307D4401A02D3EFF3F7
:10083000008010BDEFF3008010BD081A03D3EFF362
:100840000080904305E0EFF3008001219043C90749
:10085000084380F3008810BD0D231B041A4204D006
:100860001146002000F02DF810BD00F04BF810BD2F
:1008700000000090754600F04DF8AE460500694650
:100880005346C008C000854618B020B5FFF796FC57
:1008900060BCB64600260027C0C5C0C5C0C5C0C5DF
:1008A000C0C5C0C5C0C5C0C5403D490849008D464A
:1008B000704710B50446C046C0462046FFF751FCBD
:1008C00010BDC80212D54803400F002804D0C80349
:1008D000C043012188407047EFF300800001000908
:1008E00003210907084380F3008870470020704700
:1008F00010B500200249029A00F010F810BD000067
:100900000000F87F10B5024800F008F810BD0000A4
:100910000000C07F004870479000002010B50C46D2
:100920001107090F092904D00A290AD008290CD176
:1009300004E011460820FFF7C4FF06E0510606D583
:1009400001E0510601D50120C007214610BDD106A6
:1009500007D501010909CC084907000E0006044328
:1009600009E0410F20024907000A0143200E00065A
:100970001D22D14101430846E7E700000149182044
:10098000ABBEFEE726000200704770B514460D4668
:100990000646200407D0B0B200F006F82870641EA6
:1009A0006D1C761CF5E770BD70B5044600F0F0F8DC
:1009B000A020214DA847214EB047200AA847B047A4
:1009C000E0B2A847B04700F0E3F8A120A847B0473D
:1009D000002000F057F9044600F0FAF8204670BDF8
:1009E00070B514460D460646200407D02978B0B2EB
:1009F00000F006F8641E6D1C761CF5E770BD000063
:100A0000F8B50C46054600F0C3F8A0200A4EB047E2
:100A10000A4FB847280AB047B847E8B2B047B847C6
:100A20002046B047B84700F0D3F80A20F8BC02BC13
:100A30008E4600F09BB8C046E90C00084D0D00083A
:100A4000FCB5491E0023009301919AB2914212DD38
:100A50008C1A009DAAB294420ADD5200875A861869
:100A60007288974202D9B11C0F8032806D1CF1E769
:100A70005B1C0199E9E7FCBD80B500F011F800F0BE
:100A8000D3FE00F0ABFF00F037FF00F07BFE00F07C
:100A900009FF00F02FFE80BC01BC864600F062BF5B
:100AA000F8B50020022101F0F1FB0A2000F05EF809
:100AB000694D287941196F268C5D00F0B7F88442A2
:100AC00008D17020285C000229467031497840180E
:100AD000286301E00120687101240221204601F011
:100AE000D5FB0A2000F042F8287941198F5D00F00B
:100AF0009DF8874208D17020285C00022946703199
:100B000049784018686300E06C711320022101F0FD
:100B1000BDFB0A2000F02AF8287941198E5D00F00B
:100B200085F8864208D17020285C00022946703181
:100B300049784018A863F8BD6C71F8BD702246482A
:100B400000217A2A02D08154521CFAE78170018078
:100B50007047C04634480021417070473248002138
:100B600081707047304800210170704781B000905B
:100B700003480099016001680029FCD101B0704769
:100B8000AC05002081B00090009801B070470000D3
:100B9000F8B501F067F8EB4C01262046314602F02B
:100BA000B6FA02252046294602F0B1FA0427384653
:100BB000FFF7E8FF2046314602F0A7FA3846FFF774
:100BC000E1FF20462946F8BC04BC964602F09DBAD7
:100BD000F8B501F047F8DB4C02252046294602F023
:100BE00094FA01262046314602F08FFA042738464F
:100BF000FFF7C8FF2046294602F089FA2046314611
:100C000002F085FA3846F8BC02BC8E46FFF7BABF40
:100C1000054840787047C046034880787047C04612
:100C2000014800787047C0461C010020B0B5401E46
:100C30000021094B70240A46CDB2A84204DD5D199B
:100C40002D5D5219491CF7E70C4801788918407846
:100C50000918FF208843B0BD4801002010B5401E90
:100C60000021064B0A46CCB2A04203DD1C5D1219DE
:100C7000491CF8E7FF20904310BDC046B005002096
:100C8000FEE70000FEB5009000F0E6FF002102261E
:100C9000012001900C46019D07291CD8BD4F384604
:100CA0000291314602F031FA3046FFF76BFF3846C9
:100CB000314602F02CFA3846294602F02CFA274633
:100CC00004462846FFF75EFF0299601E84417800C3
:100CD0000419491CE0E7009810B100F07FFF01E023
:100CE00000F09CFFE0B2FEBDFEB5044600F0BAFF86
:100CF000A8480226314602F008FA00270120019098
:100D0000072F1FD860B200280294A24D284603D4B2
:100D1000019902F0FAF902E0019902F0F8F930467F
:100D2000094CA0472846314602F0F1F93046A04769
:100D30002846314602F0E9F93046A0477F1C029C64
:100D40006400DDE7FEBDC046850B000870B500F00D
:100D500083FF904C0221204602F0D9F90125284654
:100D6000FFF710FF00262046294602F0D4F930B1E3
:100D7000701CFA2E0646F6D3FFF72AFF04E0022184
:100D8000204602F0C2F90025284670BDF8B5E74CB0
:100D9000204602F0ABFD601C02F0A8FD0920C7064A
:100DA00000240125E24E3846294622462B46B0470C
:100DB00003263846214632462B4602F0D0F9384603
:100DC000294602F0A2F9DD4F38462946224644F270
:100DD0000003D74DA84738462146324644F2000367
:100DE00002F0BDF9384644F2000102F090F93846AD
:100DF0002146224641F20003A847F8BD00F066B83C
:100E0000FEB5CA4802F072FD0920C6060121019113
:100E10000025202730462A463B46C54CA0470322E2
:100E20000292C44C304629463B46A04730463946DC
:100E3000C14A90471027304601992A463B46BC4C90
:100E4000A04730462946029A3B46BA4CA047304656
:100E50003946B94A90474027304601992A463B46D1
:100E6000B34CA04730462946029A3B46B14CA047B6
:100E700030463946B04A90478027304601992A4685
:100E80003B46AB4CA04730462946029A3B46A94C0C
:100E9000A04730463946A84A9047A44802F026FDAC
:100EA000A64E3046019C21462A462346A04FB8470D
:100EB00030462946029A23469E4DA8473046214691
:100EC0009D4A03B0F0BC08BC9E461047F8B51B48CD
:100ED00002F00CFD1A4801250024954E29462246B1
:100EE00042F20003B0470326924F1548214632468E
:100EF00042F20003B847124842F2000102F005F93D
:100F00000E48C01C02F0F2FC2248294622462B461D
:100F1000874FB8471F48214632462B46854FB84772
:100F200002271C48294622463B46814DA8471948BE
:100F3000214632463B467F4CA047F8BD13050000D2
:100F40000008004800140048F8B5784C204602F02C
:100F5000CDFC601D02F0CAFC0E4E0024012580234A
:100F6000734F304621462A46B84740233046214633
:100F70002A46B8470920C606304621462A4641F28D
:100F80000003B847304621462A4640F20013B847CE
:100F9000F8BDC04600140048B0B50D4802F0A6FCEC
:100FA000664C0121002520462A4640F6000302F047
:100FB000B7F803222046294640F6000302F0CFF896
:100FC000204640F60001B0BC04BC964602F09DB835
:100FD0001205000070470000FEB5DC4802F086FCF8
:100FE0000920C70601260024514D384631462246C5
:100FF00048F20003A847032202924E4D384621468C
:1010000048F20003A847384648F200014A4A904790
:10101000CE48401C02F06AFC484F384601963146E3
:10102000224640F20023424DA84738462146029D01
:101030002A4640F200233F4FB847404F384640F21F
:1010400000213D4A904738463146224640F200137F
:10105000374FB847394F384621462A4640F20013E9
:10106000344DA847384640F20011334A9047802556
:101070003846314622462B462D4FB8472F48214649
:10108000029A2B462B4FB8472C4F384629462A4AFE
:10109000904740253846314622462B46244EB047DD
:1010A00038462146029A2B46224EB04738462946FA
:1010B000214A904720253846019F394622462B4633
:1010C0001B4EB0471D482146029A2B46194EB04789
:1010D0001A4E30462946184A904710253046394660
:1010E00022462B46124FB84730462146029A1646F2
:1010F0002B46104FB8471148074629460E4A9047DD
:1011000008253846019922462B46094FB8470B4817
:101110000746214632462B46064CA047384629460C
:10112000054A03B0F0BC08BC9E46104711050000FC
:10113000213100085F3100080B310008000400482D
:101140000C48006840F2E831B0FBF1F0401E010E9F
:1011500000D0FEE70849094A5060094803680B407F
:101160000321890759180160002090600720106052
:101170007047C04608000020FFFFFF0010E000E0BD
:1011800020ED00E0F0B587B0354940F210608847A7
:10119000344D35492846884703AC344920468847B2
:1011A0004720029020803248059000200190049052
:1011B000304A28462146904701272F4A284639467B
:1011C00000979047142002212C4A90472C4928462A
:1011D000884740F21060401C21498847294E30461C
:1011E0002149884703AD284620498847029828802E
:1011F0001F480590019C0494304629461D4A90479B
:10120000304639461C4A90471520032529461B4A7B
:10121000904730461A49884740F21060801C1049B8
:101220008847194E30461049884703AF38460F4962
:101230008847029838800E48059004943046394615
:101240000C4A9047304600990B4A90471620294691
:101250000A4A904730460A49884707B0F0BDC04661
:10126000ED38000800400140313900087D3A00089F
:10127000E7030000A5390008593A0008F1360008D4
:101280009B3900080044014000480140FEB502902F
:101290001C200225294602F02BFA2C4802F026FBDE
:1012A0000920C70601240426019638462146324605
:1012B00001F000FF384629462246334601F030FF50
:1012C0000021009138462246334601F048FF0826A7
:1012D00038462146324601F0EDFE38462946224680
:1012E000334601F01DFF3846009F394622463346FB
:1012F00001F035FF164802F0F9FA164D284602F0C3
:1013000013FC2846029902F0DDFB2846394602F01C
:101310007DFC284641F2000102F08DFC284640F297
:10132000004102F05EFC2846019902F067FC284665
:10133000314602F078FC284602F010FC05212846D0
:1013400003B0F0BC04BC964602F01EBC11050000C0
:101350001107000000440040F8B500F07FFF0A24A8
:101360000F4E2046B04700F049FF2046B04700200E
:1013700002250C4A0C4F2946B8472046B0470120A9
:1013800029460246B8471320084A2946B84720464E
:10139000B04700F04BFFF8BC01BC864600F008B82F
:1013A0006D0B0008040A0000B1220008650400006B
:1013B000FEB570240221204600F068FF3220FFF7BE
:1013C000D5FBEA4E307981196F254F5DFFF72EFC72
:1013D000874206D1305D00023146703149784018AD
:1013E000B0607120022100F051FF3220FFF7BEFBF8
:1013F000307981194F5DFFF719FC874206D1305DC6
:1014000000023146703149784018F06072200221A4
:1014100000F03CFF3220FFF7A9FB307981194F5DC6
:10142000FFF704FC874206D1305D0002314670317F
:101430004978401830617320022100F027FF3220E4
:10144000FFF794FB307981194F5DFFF7EFFB87427F
:1014500006D1305D00023146703149784018706124
:101460007420022100F012FF3220FFF77FFB307959
:1014700081194F5DFFF7DAFB874206D1305D00022C
:101480003146703149784018B0617520022100F072
:10149000FDFE3220FFF76AFB307981194F5DFFF7BF
:1014A000C5FB874206D1305D000231467031497874
:1014B0004018F0617620022100F0E8FE3220FFF7AC
:1014C00055FB307981194F5DFFF7B0FB874206D19C
:1014D000305D000231467031497840183062772023
:1014E000022100F0D3FE3220FFF740FB3079811952
:1014F0004F5DFFF79BFB874206D1305D000231460E
:1015000070314978401870620221284600F0BEFE12
:101510003220FFF72BFB307981194D5DFFF786FBF9
:10152000854208D1305D000231467031497840185B
:101530000290B06201E0B06A0290B0680190374654
:101540000C37BCCF306A0090716A01988218D218AB
:1015500012195219D219009810184018401E80B262
:1015600003494140F1620298091A48424841FEBDD0
:10157000FFFF0000024840F6000101F0CABDC0466E
:10158000000400487047704780B5FFF745FB30B155
:10159000FFF7F0FF80BC01BC8646FFF7DFBA80BDD5
:1015A000F8B50024334E0C27334B204631463A46DB
:1015B0009847324831463A46FEF712FE30483146E7
:1015C0003A46FEF70DFE06252D482946FFF738FA64
:1015D000242031463A46284B98472A4831463A4615
:1015E000FEF7FEFD284831463A46FEF7F9FD26484B
:1015F00000952946FFF724FAAC2031463A461E4BA7
:101600009847224831463A46FEF7EAFDC02540F2A7
:10161000021031462A46184FB8471D4831462A461F
:10162000FEF7A6FD1B48602531462A46B8471A4FEB
:10163000384631462A46FEF79BFD40F2E830602CE2
:1016400014D03959491C00D1385139194A68521CF3
:1016500001D100224A608A68521C00D18860CA68A1
:10166000521C01D10022CA601034E8E70B480099EF
:101670000170F8BD100400208B0900080201002051
:101680000E0100202C030020A005002038030020BC
:1016900050030020DE020000CC020020C80200201F
:1016A00070B5114C8021114E2046B047104D287066
:1016B00040212046B04768700920C406204641F208
:1016C0000001B047A870204640F20011B047C000AA
:1016D000A9788900014368784000084329780143CC
:1016E0000F20884370BDC04600140048CF1B00087F
:1016F0004401002070B52220022100F0C7FD0A201D
:10170000FFF734FAD44E307981196F228C5CFFF7E1
:101710008DFA84420AD17020305A000400BAFFF7D3
:1017200023F8FEF703FF04460D4603E00120707125
:1017300000242546B06E0E4902F092FD08B90E4A0B
:1017400000E00C4A08B90E4B00E00C4B204629463D
:10175000FEF7C8FDFEF788FDF066306D3F210906F3
:1017600002F073FD08B90020F06670BD480100204A
:1017700000005C42CFF753E34E621058A59BB43F84
:1017800039B4B83F70B52820032100F07FFD0A204E
:10179000FFF7ECF9B04D287941196F240E5DFFF782
:1017A00045FA86420BD17020285C0004294670312E
:1017B0004A781202101889784018686501E0012003
:1017C00068710220014600F061FD0A20FFF7CEF9A2
:1017D000287941190C5DFFF729FA844208D170205D
:1017E000285C00022946703149784018A86501E05C
:1017F00001206871686DFEF7B7FF0446286AFEF79E
:10180000B3FF0146204602F003FE3121090602F033
:10181000FFFD934C214602F0FBFD2146FEF7B0FE92
:10182000E865286670BDC046B0B52420032100F0ED
:101830002DFD0A20FFF79AF9874D287941196F226B
:101840008C5CFFF7F3F984420BD17020285C000414
:10185000294670314A781202101889784018E863D6
:1018600002E001206871E86B010218D4FEF77CFFEA
:101870000446A868FEF778FF0146204602F0C8FD3E
:101880000D21890602F0C4FD754C2146FEF778FE55
:10189000214602F0BDFD2146FEF772FE00E0002069
:1018A0002864B0BDB0B52320022100F0EFFC0A206F
:1018B000FFF75CF9684C207901196F228D5CFFF706
:1018C000B5F9854208D17020205C000221467031B4
:1018D0004978401802D1B0BD01206071FEF744FF85
:1018E0004121090602F094FD01460248FEF748FE38
:1018F0006066B0BD647A5A4AB0B52C20042100F06D
:10190000C5FC0A20FFF732F9534D287941196F229F
:101910008C5CFFF78BF9844203D1286F00BAE8642E
:1019200002E001206871E86C0121CA0700219042A1
:1019300000D9C9434840FEF717FF04466869FEF71F
:1019400013FF214602F064FD0321090702F060FD48
:10195000434C214602F05CFD2146FEF711FE28654E
:10196000B0BDC04670B52720032100F08FFC0A20CF
:10197000FFF7FCF8384E307981196F228C5CFFF745
:1019800055F984420AD17020305C00043146703130
:101990004A78120210188978441801E00120707109
:1019A000306DFEF7C3FD0A4A0A4B02F043FC0546C0
:1019B0000120C1058C4201D90006041B2046FEF718
:1019C000D3FE0549FEF7DCFD05B10020B06670BD11
:1019D000333333333333D33FFEFFFF4AB0B52620D2
:1019E000032100F053FC0A20FFF7C0F81A4D2879B4
:1019F00041196F228C5CFFF719F984420BD17020DA
:101A0000285C0004294670314A781202101889783F
:101A10004018686402E001206871686C010218D403
:101A2000FEF7A2FE04462869FEF79EFE0146204608
:101A300002F0EEFC6921C90502F0EAFC0749FEF755
:101A40009FFD074C214602F0E3FC2146FEF798FD7E
:101A500000E00020A864B0BD480100200000C8429A
:101A600000007A4480B547480078C007564840F2E5
:101A7000002106D101F049FB434800780121884349
:101A800005E001F044FB40480178012008433E494D
:101A9000087080BD80B53B488078C0074A4840F256
:101AA000001106D101F031FB3748807801218843CD
:101AB00005E001F02CFB34488178012008433249CD
:101AC000887080BD80B52F480079C0073E4807D197
:101AD000802101F01AFB2C4800790121884306E09F
:101AE000802101F014FB2848017901200843264990
:101AF000087180BD80B523488079C007324807D17E
:101B0000402101F002FB204880790121884306E052
:101B1000402101F0FCFA1C488179012008431A4950
:101B2000887180BD80B51748007AC007264807D164
:101B3000202101F0EAFA1448007A0121884306E0E6
:101B4000202101F0E4FA1048017A012008430E49EF
:101B5000087280BD80B50B48807AC0071A4807D14B
:101B6000102101F0D2FA0848807A0121884306E06A
:101B7000102101F0CCFA0448817A0120084302497F
:101B8000887280BD380300204403002070477047EE
:101B900010B50D4C204644F2000101F0B6FAFFF7F3
:101BA00061FFFFF777FFFFF78DFFFFF7A3FFFFF759
:101BB000B9FFFFF7CFFF204644F2000110BC04BC80
:101BC000964601F0A4BAC04600040048704780B5AC
:101BD00001F0A1FA411E884180BD000070B52D4C76
:101BE00002250D4E20462946B04700F03BF8012162
:101BF0002046B0472846FEF7C5FF2046294601F09B
:101C000086FA2846FEF7BEFF20462946324670BCBB
:101C100008BC9E461047C0460B310008B0B51D4CAD
:101C200002252046294601F070FA00F01BF8012138
:101C3000204601F06CFA2846FEF7A4FF204629460C
:101C400001F065FA2846FEF79DFF20462946B0BC04
:101C500004BC964601F059BA0E48002101230A46F9
:101C600001F05EBA70B50B4C0025012620463146C6
:101C70002A46334601F054FA0322204629463346C9
:101C800001F06DFA8021204670BC04BC964601F03C
:101C90003EBAC04600140048F8B504460027094D76
:101CA0000A4EA7420CD00848C15D284601F036FF15
:101CB0002846314601F057FF0028F9D07F1CF0E795
:101CC000F8BDC04600440040B005002006070000F3
:101CD0000348016811B10168491E01607047C046A0
:101CE000AC05002030B43348026801210A43026089
:101CF00002689207FCD542682F4B1340436042684C
:101D00002E4B1340436002682D4B13400360C26AA0
:101D10000F239A43C262026B40F203139A43026399
:101D20000A04036B93430363CA07036B9343036380
:101D3000426B8A4342630022826002680A43026067
:101D4000204B022204685D1E9D4202D214402B46A5
:101D5000F8D003689B0700D4FEE71B4B1C680725DF
:101D6000AC431C601C6814431C60436843604368B8
:101D70004360436843604368144C1C4044604368BC
:101D8000134C1C4344600B0604681C430460036846
:101D90009B01FCD543680324A3434360436813437A
:101DA000436042681207FCD5C806002130BC01F030
:101DB000D3BCC046001002400C00FF08FFFFC277F2
:101DC000FFFFF2FEFF04000000200240FFFFC2F709
:101DD0000000040810B50A4C0121204601F044FE21
:101DE00068B10121204601F03BFE0021204601F0B0
:101DF0009DFD0448006810BC02BC8E46004710BD23
:101E00000020004024020020F8B59C4D0124284603
:101E1000214601F029FE012803D10121284601F0C5
:101E20001FFEB84FB888401CB88081B2814200D0F4
:101E300023E10022BA80F868401CF8603969002963
:101E4000009200D18AE08E4D29888E4E884203D0C0
:101E50008D4A914200D061B9304644F2000101F050
:101E600054F9FFF7FFFD304644F2000101F04FF94D
:101E7000F8686988884203D0834A914200D061B9EA
:101E8000304644F2000101F040F9FFF703FE30460E
:101E900044F2000101F03BF9F868A988884203D0B8
:101EA000794A914200D061B9304644F2000101F014
:101EB0002CF9FFF707FE304644F2000101F027F944
:101EC000F868E988884203D06F4A914200D061B92E
:101ED000304644F2000101F018F9FFF70BFE3046DE
:101EE00044F2000101F013F9F8682989884203D00F
:101EF000654A914200D061B9304644F2000101F0D8
:101F000004F9FFF70FFE304644F2000101F0FFF83C
:101F1000F8686989884203D05B4A914200D061B970
:101F2000304644F2000101F0F0F8FFF713FE3046AE
:101F300044F2000101F0EBF8F868544949898842FD
:101F400005D05148814202D0002900D094E04B488E
:101F500001F01EFD0098F86038618DE07969002974
:101F600000D189E04A4D2988464E884203D0464A2E
:101F7000914200D061B9304644F2000101F0C5F849
:101F8000FFF770FD304644F2000101F0C0F8F86838
:101F90006988884203D03C4A914200D061B93046FA
:101FA00044F2000101F0B1F8FFF774FD304644F24D
:101FB000000101F0ACF8F868A988884203D0324AE1
:101FC000914200D061B9304644F2000101F09DF821
:101FD000FFF778FD304644F2000101F098F8F86808
:101FE000E988884203D0284A914200D061B930463E
:101FF00044F2000101F089F8FFF77CFD304644F21D
:10200000000101F084F8F8682989884203D01E4A4B
:10201000914200D061B9304644F2000101F075F8F8
:10202000FFF780FD304644F2000101F070F8F868D7
:102030006989884203D0144A914200D061B9304680
:1020400044F2000101F061F8FFF784FD304644F2EC
:10205000000101F05CF8F8680E494989884205D012
:102060000948814202D00948408928B9034801F053
:102070008FFC00987861F8603C70F8BD004001402A
:102080002C03002000040048FFFF0000A0050020F2
:10209000020100200E010020B0B50B4D012428469E
:1020A000214601F0E1FC012803D10121284601F07D
:1020B000D7FC1448C188491CC18089B2642902D365
:1020C00044700021C180B0BD00440140B0B50C4D4A
:1020D00001242846214601F0C7FC012803D1012133
:1020E000284601F0BDFC07480189491C018109B25D
:1020F00040F2E832914202DB847000210181B0BDE0
:10210000004801401C010020B0B51D4C354D204653
:10211000294601F057FD30B11A4800688047204633
:10212000294601F03BFD184D2046294601F04AFDA5
:10213000012806D11348006880472046294601F04F
:102140002DFD124D2046294601F03CFD30B11048CE
:10215000006880472046294601F020FD0D4D2046AD
:10216000294601F02FFD48B1094800688047204604
:102170002946B0BC04BC964601F010BDB0BDC046B7
:10218000003801401C020020000203070700070777
:102190002002002006000607B0B5114C114D204664
:1021A000294601F00FFDD0B12046294601F0F6FC8A
:1021B0000D4800780D4D297881420BD2204601F060
:1021C000A9FC29780B4A50540B4801220270481C84
:1021D0002870B0BD00202870054801210170B0BDF5
:1021E00000440040050005074C0100204A01002082
:1021F00049010020B801002048010020B0B53F4847
:10220000002101710424C4703B4D5A20A870EA20BB
:102210006870A52028702046FEF720FDE870204653
:10222000B0BC02BC8E46FFF737BDC046B0B53348E0
:10223000002101710424C4702F4DDC20A870EA2015
:102240006870A52028702046FEF708FDE87020463B
:10225000B0BC02BC8E46FFF71FBDC046B0B52748D4
:10226000002101710424C470234DE520A870EA20E8
:102270006870A52028702046FEF7F0FCE870204624
:10228000B0BC02BC8E46FFF707BDC04610B51A4A67
:102290005070A5201070194C0220E070481C20716D
:1022A000FEF74CFCE07810BC02BC8E46FFF7F4BC95
:1022B000BCB5114BA5241C70802404435C700092B3
:1022C000981C6A46521E0C4624B1155D0570401CD0
:1022D000641EF9E7094800220271C91CC170CCB222
:1022E000E018451E2046FEF7B9FC28702046BCBC0D
:1022F00002BC8E46FFF7D0BCB0050020480100208C
:10230000B0B50020064CA047064D28600120A0472C
:1023100068600220A047A8600320A047E860B0BD25
:10232000C537000834010020F0B55448001D544959
:1023300008310022534BBF240C2A0FD09D5CAE06FF
:1023400006D50E680768B74202D94026354300E03B
:1023500025409D5420311830921CEDE74A48062153
:102360000170F0BDF0B545480830454918310122EB
:10237000444BFB240D2A0FD09D5CAE0706D50E689A
:102380000768B74202D90426354300E025409D5432
:1023900020311830921CEDE73B4806210170F0BD5A
:1023A000F0B536481030364910310022354EFE2344
:1023B0000C2A17D0B556002D04D4B41865781D40EA
:1023C00065700BE0B5186E780F680468BC4202D9DE
:1023D0000124264300E01E406E702A4E2031183042
:1023E000921CE5E7284806210170F0BD80B500F099
:1023F00029F800F009F8FFF797FFFFF7D1FF80BC3D
:1024000001BC8646FFF7AEBFF0B51D48001D002198
:102410001A4A1C4BEF240C290FD05D5C2E0706D501
:1024200006681768B74202D21026354300E02540FF
:102430005D5420301832891CEDE7134806210170E5
:10244000F0BDC046F0B500200C490D4A0D4BFB24F1
:102450000C280FD01D5CAE0706D516680F68B74272
:1024600002D90426354300E025401D54203218319E
:10247000801CEDE7044806210170F0BD3802002001
:102480005003002038030020C802002010B5144675
:1024900008463F490A220A700722214601F076FDCC
:1024A000012804D1044801F0EBFD012801D00320EC
:1024B00010BD002010BDC046204E0000F8B50646F5
:1024C0000F4CA088000A16D1A0880527032810D336
:1024D0000D460092A188264801F068F948B92449C0
:1024E00008783070481C2860A088801E00990880F9
:1024F00000273846F8BD03A00C499C22FFF7C6FF11
:10250000C401002075735263764275666665725029
:102510006F73203C204D425F5345525F5044555FDE
:1025200053495A455F4D4158000000001C480008BF
:10253000B0B5174D6B780BB1052516E00124EC8082
:102540004B1EAB601870E8888018E880E988184650
:1025500001F02CF9E9884A1CEA80054A5054AC7015
:1025600000252846214601F073FB2846B0BDC04631
:10257000BA05002010B501200024214601F068FBB7
:1025800003484470204610BC02BC8E4601F0ECBCEF
:10259000C401002080B50020014601F059FB80BC39
:1025A00001BC864601F088BB10B5064C2078012896
:1025B00005D10548806880470020207010BD0620A6
:1025C00010BDC0460C00002004020020F8B50C46E7
:1025D0000988032505292FD10279C17809028E18AF
:1025E000711E89B2314B994226D8811C009187789F
:1025F0004178002525800123037023885B1C2380FC
:102600005307B2B2D60803B1761C009B46702088EF
:10261000401C20800802C019401C81B218462B467D
:1026200000F0E8FA20B1F8BC02BC8E4601F09EB87A
:10263000F0B22188081820802846F8BDF8B50C466D
:102640000988032505292ED10279C17809028E183F
:10265000711E89B2154B994225D8811C009187784B
:102660004178002525800223037023885B1C23808A
:102670005307B2B2D60803B1761C009B467020887F
:10268000401C20800802C019401C81B2184600F08E
:1026900001FB20B1F8BC02BC8E4601F067B8F0B275
:1026A0002188081820802846F8BDC046CE070000C3
:1026B000F8B50C4609880325052923D10279511E56
:1026C0007C291FD8831C8178477800252580032624
:1026D00006702688761C2680560046702088401C8E
:1026E000208038024018401C81B218462B4600F06A
:1026F000F7FA20B1F8BC02BC8E4601F037B820884A
:10270000801920802846F8BDF8B50C4609880325B5
:10271000052928D10179C278120251184A1E92B2B5
:102720007B2A20D8821C0092877843780025258058
:10273000042202702288521C22808AB256004670FF
:102740002088401C20801802C019401C81B20098CB
:1027500000F096FC20B1F8BC02BC8E4601F006B831
:102760002088801920802846F8BDF8B505460888DD
:102770000A2841D30C462879E97809020F18781EF7
:1027800080B203267C2838D8287AE979090208180B
:10279000411E89B2782930D8697A82B250008142CC
:1027A0002BD1A879697909020818411CA8780090F2
:1027B0006E7828460A3089B2012300F091FAB0B948
:1027C000BAB2300200994018411CA81C002626808D
:1027D00017232B7023885B1C238057006F7023887E
:1027E0005B1C238089B2334600F07AFA38B1F8BC1A
:1027F00002BC8E4600F0BABF00263046F8BD2088E5
:10280000C0192080F9E70000B0B50C4605490D88D5
:10281000401C891C2A46FDF7E3FC681C2080002030
:10282000B0BDC046D40100201CB509880324052989
:102830001AD10179C1B982784378C178FF2900D0D3
:1028400091B918028018421C01A800244470FF3975
:102850004B424B41037091B20122134600F0CAF97A
:1028600010B100F083FF044620461CBD80B50988E6
:10287000052910D18178427812025118491C89B279
:10288000C01C0122134600F02BFA30B180BC02BC00
:102890008E4600F06BBF032080BD002080BD70B568
:1028A0000C460A880321062A24D30679C27812022C
:1028B0009519AAB2D308760700D05B1C6D1EADB285
:1028C0002D097A2D16D84579DBB29D4212D1817837
:1028D00043781B025918491C89B2801D012300F05E
:1028E00089F920B170BC02BC8E4600F03FBF0520C4
:1028F00020800021084670BDB0B50C460A8803212F
:10290000062A20D30279437955062D0EAB421AD1FF
:10291000C3781B029A18531E9BB2772B13D8817869
:1029200043781B025918491C89B2801D92B20123B9
:1029300000F0D6F920B1B0BC02BC8E4600F016BF44
:102940000520208000210846B0BD0000F8B50546EE
:10295000022091B3CC081E2C2FD8069C524E317009
:10296000012D15D04DBB254D2548264FB760F06091
:102970003561214870611F48B0611D48F0611B48F6
:102980003062084611461A46234600F091F813E0DB
:10299000134D1448144FB760F06035610F487061F3
:1029A0000D48B0610B48F061094830620846114695
:1029B0001A462346FFF76AFD00B1F8BD01F0CEFAD2
:1029C00020B13848012101700020F8BD0320F8BD76
:1029D000253E00085D3E0008193D0008BD240008A2
:1029E0003125000895250008752500086941000873
:1029F000B5410008D9400008ED2A0008612B000805
:102A0000E12B0008C52B00087CB52648007808B1EA
:102A1000062445E001A801F095FA002401283FD1E1
:102A200001A80078022812D0012839D11E4D6B6907
:102A3000681C294624312A1D984788BB6878297864
:102A4000884200D060BB022001F08EFA28E0164DCB
:102A50006A6A1178A97000230120144C802B0AD0D7
:102A6000E65C46B18E4201D00833F7E7E0184368D0
:102A7000291D104698476978002489B158B1012171
:102A8000A980A97880220A43696A0A70A9884A1C29
:102A9000AA806A6A5054AA88696A28782B6998477C
:102AA00020467CBD0C000020040200201000002005
:102AB00010B5144608460822214601F067FA01289D
:102AC0000ED144F60030844201D9232003E0600097
:102AD0000549B1FBF0F080B201F0D2FA012801D033
:102AE000032010BD002010BDA07F1700F8B50646DA
:102AF0000F4C6088800A16D160880527042810D3FF
:102B00000D46009261882E4800F0C2FF48B92C495A
:102B100008783070481C28606088C01E00990880C2
:102B200000273846F8BD03A00C499C22FFF7AEFCF5
:102B3000F8010020757352637642756666657250BF
:102B40006F73203C204D425F5345525F5044555FA8
:102B500053495A455F4D4158000000009D48000808
:102B6000B0B51E4D2B78012B26D10124AC804B1E15
:102B7000AB601870A8888018A880A988184600F053
:102B800087FFA9884A1CAA800D4A5054A9884B1C6B
:102B9000AB80000A5054A868007801F067FAA88852
:102BA000401EA880A868401CA8606C7000252846BC
:102BB000214601F04DF800E005252846B0BDC0468D
:102BC000BA05002080B5054800210170012001F000
:102BD0003FF880BC01BC864601F086B8F8010020B1
:102BE00080B50020014601F033F880BC01BC864668
:102BF00001F062B8FEB514460246491E88B20019BB
:102C0000042824D8601E0825019590FBF5F0451C8A
:102C10000020F3B1012B1BD100901D4B280435D0AF
:102C20006D1E029210782246019F541E12040BD092
:102C30003A0609D0012202408EB29A55491C7F1EE5
:102C4000C0B240082246F0E7029A521CE6E7012093
:102C5000FEBD0090082001900D4F280416D002926E
:102C60006D1E002622460198541E12040AD0020648
:102C700008D08AB2BA5CB2401343761C491C401E8D
:102C80002246F1E7029A1370521CE6E70098FEBD57
:102C9000BA090020F0B5491E8BB2DC0801217D2C59
:102CA0001BD39B1840F2EC34A34216D8511E0823C4
:102CB00091FBF3F14C1C002125040ED0641E164636
:102CC0001D46721E360404D06F1E2D0616463D4664
:102CD000F7D100250570401CEEE70846F0BD000066
:102CE000FEB50646481E87B2780901257D2800D228
:102CF000BBE01446B818CA4A904200D9B5E040F685
:102D0000AB703A1A0B32C74842600025012B10D035
:102D1000002B00D0A9E00292C048421C97424ED13D
:102D2000012C4CD102984000D4490988BF4A115265
:102D3000C8E00292019544700322D24340F2D0735E
:102D40005343BA48C3187D005B1925462A0409D0AD
:102D5000327812021A80707810181880B61C9B1CEA
:102D60006D1EF3E741F2EB10081A563080B20628C8
:102D700047D841F2EA103E1A5636AA4806708660D5
:102D800002984000A9490F18F0B24000B549081850
:102D90002106CD0D39462A46FDF722FAA74C2046DA
:102DA00039462A46FDF71CFA7004000C21462A46D3
:102DB000FDF716FEAC4D0C222846AA494EE041F222
:102DC00072028A1AC63292B2482A50D896497918A5
:102DD0000C2291FBF2F19348017002984000934A53
:102DE0001018C9B218224A43A24989186200FDF797
:102DF000F7F98A480C30874264D19F48012101606D
:102E000060E08B4843181846443080B206286CD8DE
:102E100041F2EA103E1A44368248067086600298F3
:102E2000400082490F18F0B240008C490818210672
:102E3000CD0D39462A46FDF7D3F9804C2046394658
:102E40002A46FDF7CDF97000243080B221462A468B
:102E5000FDF7C6FD824D0C2228468049FDF7C0F9DA
:102E600006212846FDF7ECFD019D2846FEBD7F4A60
:102E70008A1892B2062A25D87239CAB252007C4BFF
:102E800001959D5C012028406F4DAB5C0093FE25B1
:102E9000009B1D402B18764DAB5462480170A91859
:102EA0004B78F8251D406848821852780723134054
:102EB0005A19019D4A70029840005C4A101862003D
:102EC000FDF78EF90320C04340F2D07141435748CB
:102ED0004018790040182104C7D04178317001783A
:102EE0007170B61C801C641EF5E798B206282ED8B7
:102EF00041F2EA103F1A4B48077087600298400081
:102F00004A490E18F8B240004F4908182106CD0D65
:102F100031462A46FDF764F9484C204631462A4698
:102F2000FDF75EF97800AC3080B221462A46FDF705
:102F300057FD3C4840780628019D61D142494878B8
:102F40000978C9075AD1C0065AD543485CE041F216
:102F50000430081AEE3080B2602823D841F20330E2
:102F60003F1AEE372F498F60102097FBF0F0087062
:102F7000029949002D4A5618C0B24001314908183B
:102F80002106CD0D31462A46FDF72AF92B4C204665
:102F900031462A46FDF724F9780040F2FE11401828
:102FA000FC3825E02348081880B2302800D95BE7B8
:102FB00041F203303F1A1B498F60082097FBF0F065
:102FC000087002994900194A5618C0B200011A49FE
:102FD00008182106CD0D31462A46FDF701F9174C98
:102FE000204631462A46FDF7FBF878001449401880
:102FF00080B221462A46FDF7F3FC35E7000702D4EC
:10300000FEF7C6FD31E7114801210160104800F0CC
:10301000C4FC10480025056027E7C0469F0F00004C
:10302000881300002C02002055F0FFFFBE0900208D
:1030300015EE0000FCEC0000CC020020D8040020BB
:10304000DE02000050030020380300203001002081
:1030500000400140280100202C0100202C0300200A
:10306000A0050020020100200E0100208EEF0000CC
:103070004403002038020020F80000200000002057
:1030800010B50346481E81B20120084CA1420BD363
:103090008918074CA14207D80020110404D05870A9
:1030A00018709B1C521EF8E710BDC046B80B0000FC
:1030B000BC0B0000FCB50191016A0090446A002538
:1030C0002E46202D0CD01746F740FF0705D0019F54
:1030D000AF400F23AB40994339432D1D761CF0E7D9
:1030E00008250026202E0CD01346EB40DB0705D028
:1030F000019BB3400F27B740BC431C43361D6D1CDA
:10310000F0E7009801624462FCBD81627047816112
:103110007047C162704700690840411E884170478E
:10312000FEB50293019202680090C56800263746FA
:10313000202E10D0029BFB40DB0709D0019BB3403F
:103140000324B440A5431D430B46B340A2431A4396
:10315000B61C7F1CECE700980260C560FEBDF8B5A8
:10316000012902D14168194301E041689943416056
:1031700000908168002403202646202C0CD01F4696
:10318000F740FF0705D01746A7400546A540A943CD
:103190003943A41C761CF0E700988160F8BD00005C
:1031A00086B0FEF79FFDFFF7ABF8FDF713FFEE4883
:1031B00000680C21ED4D122902D06854491CFAE731
:1031C000FDF7BEFFFDF7E2FDE94841F20001FFF720
:1031D000A2FF08B101202870FDF7DEFEFDF7B4FE66
:1031E000FDF7FAFEFDF7CEFF42F28050FEF74EF8F3
:1031F000FDF706FEFEF754FA014600220092E12098
:10320000430210460292FFF7A1FBFFF7CDF9092018
:10321000C00603902C46687801268021059140273E
:103220000496C0B2072874D8810001A251188F46B5
:1032300000F00EB800F016B800F020B800F02AB880
:1032400000F033B800F03EB800F046B800F052B8D5
:10325000C7483146FFF759FF039D28460599FFF7F8
:1032600056FF14E0C2483146FFF74FFF039D284642
:103270000599FFF74CFF2846394646E0BC483146E1
:10328000FFF743FF039D28460599FFF73EFF2846B9
:1032900039462CE0B6483146B64EB047039D284625
:1032A0000599B0472846394609E0B1483146B24E43
:1032B000B0478021039D2846B04740212846B047AB
:1032C000049E24E00121AA48FFF721FF8021039DED
:1032D0002846FFF71CFF16E00121F648FFF717FF0D
:1032E0008021039D2846FFF710FF40212846FFF765
:1032F0000EFF0CE00121EF48FFF709FF8021039D3D
:103300002846FFF702FF40212846FFF7FEFEFEF7A2
:1033100023F821466078401C6070C1B2082900D2B1
:103320007FE72746029C7C70FDF768FDFEF738F9C1
:103330007C60E44CFFF768FBFEF726F9DD4841F2BC
:103340000001FFF7E8FE002800D097E03878012858
:1033500000D193E0FDF764FC002800D183E0786899
:10336000401C7860798A884202D0A14200D069B9B5
:10337000D04D284644F20001FFF7C7FEFEF772FB6E
:10338000284644F20001FFF7C2FE7868B98A8842F5
:1033900002D0A14200D069B9C64D284644F20001CE
:1033A000FFF7B3FEFEF776FB284644F20001FFF775
:1033B000AEFE7868F98A884202D0A14200D069B98D
:1033C000BC4D284644F20001FFF79FFEFEF77AFB52
:1033D000284644F20001FFF79AFE7868398B88424C
:1033E00002D0A14200D069B9B24D284644F2000192
:1033F000FFF78BFEFEF77EFB284644F20001FFF745
:1034000086FE7868798B884202D0A14200D069B9E3
:10341000A84D284644F20001FFF777FEFEF782FB35
:10342000284644F20001FFF772FE7868B98B8842A3
:1034300002D0A14200D069B99E4D284644F2000155
:10344000FFF763FEFEF786FB284644F20001FFF714
:103450005EFE7868398D884202D0A14200D001B961
:10346000BE70FDF77FFBB878012800D062E7944872
:1034700000F08EFA0020B870786016E0FEF7F2FADD
:10348000FEF708FBFEF71EFBFEF734FBFEF74AFBD8
:10349000FEF760FBFEF77AFBFEF779FB0020B870C1
:1034A00078603870864800F073FA894C18200490D0
:1034B000FFF7AAFAFDF7ACFB002800D1F5E0787819
:1034C000072869D8810001A251188F4600F00EB874
:1034D00000F016B800F019B800F01CB800F01EB8E3
:1034E00000F029B800F031B800F048B80121714867
:1034F000FFF70BFE8021039C2046FFF708FE2DE01E
:1035000001216C48FFF701FE19E001216948FFF72E
:10351000FCFD1EE001216748684D02E0012165487D
:10352000654DA8478021039C2046A847402120469E
:10353000674CA84730E001215E48FFF7E8FD802195
:10354000039C2046FFF7E3FD21E001215948FFF7E6
:10355000DEFD8021039C2046FFF7D7FD4021204659
:103560005B4CFFF7D4FD17E004000020F0000020C2
:10357000000400480B3100080F31000801214D48BC
:10358000FFF7C5FD8021039C2046FFF7BEFD4021CB
:1035900020464F4CFFF7B9FDFDF76EFA7E78B8680C
:1035A000A8B3A6BB484C2068FDF7DEF801464748A3
:1035B000006800F02DFF05466068454C40F2E83198
:1035C000B0FBF1F0FDF7D0F80146284600F086FE8A
:1035D000FDF786F8054620603E48854205D8029BE7
:1035E0002360E36018461D4608E03B4800683B49FD
:1035F00000F00EFFFDF774F8E060029B1946782991
:1036000004D06218506295611831F8E7BB600498E5
:103610007043354605963E462718314800682F49C5
:103620000C4600F0F5FEFDF75BF838612D480068A8
:10363000214600F0EDFEFDF753F87861280122499C
:103640000C18A068FDF790F801462748006800F0C4
:10365000DFFE0546E06840F2E831B0FBF1F0FDF72F
:1036600083F80146284600F039FEFDF739F8054693
:10367000786005983018047B1C480068174900F0F2
:10368000C7FEFDF72DF80026A54200D83046B860E9
:10369000FEF7ACFE064F7878401CC1B2052900D871
:1036A00006467E70FDF756FA094CFDF76DFFFFE602
:1036B000F0000020000400480F3100080B31000822
:1036C00000400140FFFF0000CC02002090010020DC
:1036D0003802002010270000AC01002000007A44CE
:1036E000A4010020B00100208801002098010020E2
:1036F00070B540B2002817D4032302469A43144BF6
:10370000D4588507ED0EFF26AE40B4438901C9B2F7
:10371000A9402143D1501F21014001228A40400984
:1037200080000C49425070BD8207D20EFF249440A5
:103730000F230340083B0320834304481D58A5433F
:103740008901C9B291402943195070BD1CED00E0B8
:1037500000E400E000E100E0024A0A4002430248BF
:103760000260704780FFFF1F08ED00E040B10728AE
:1037700003D0012803D1022070470620704704209F
:10378000704700000A2801D2302102E0102803D23D
:1037900037210818C0B2704702A0034940F2D01286
:1037A000FEF774FE300000001C48000800220B04E5
:1037B00005D00378D218D2B2401C491EF7E7504218
:1037C000C0B27047F8B501463E4B18680C22024063
:1037D0003D48082A044618D11A689202120F0F2A8F
:1037E00001D0941C00E010241D682D0101D5113278
:1037F00014461A68D20301D4344A05E09A6A0F25A8
:1038000015406A1CB0FBF2F254431D6818681A6830
:1038100005291FD800902D062D0F2DA77F5D254669
:10382000FD409204520F2E4FBE5C2A46F2408E009D
:1038300001A080198746C04600F00AB800F011B810
:1038400000F00AB800F00EB800F00EB800F014B89E
:10385000224607E0002205E000984005400F385C52
:10386000C5402A461046F8BDD86AC0051AD4D86AA1
:10387000C00320D51C48F8BDD86A8007F2D0D86AAA
:103880000321084001282246ECD0D86A084048F2BB
:1038900000020228E6D0D86A084003280A4800D06F
:1038A0000020F8BD18680004800FD96A002904D4EC
:1038B000B2FBF0F2D6E70B48F8BD401CB5FBF0F2C6
:1038C000D0E7C0460410024000127A0000093D0013
:1038D00000000000000000000102030406070809C0
:1038E000D0470008809FD500003FAB011F21014059
:1038F00001228A4080090C494358134343507047C2
:103900001F21014001228A408009074943589343FF
:10391000435070471F21014001228A40800902491B
:1039200043581343435070470010024041627047B0
:1039300010B5154C4449884213D01449884212D01E
:10394000E849884211D03D49884213D03D49884218
:103950000DD03E4988420CD03949884213D1F63403
:1039600008E0E41D06E0F93404E0FD3402E0641DE3
:1039700000E0A41D2046FFF7CDFF204610BC02BC8E
:103980008E46FFF7BDBF10BD0B03000000100040C6
:1039900001680122914301607047016801220A43D6
:1039A0000260704710B50A888262244A904202D0B1
:1039B000234B98420BD103687024A34303604B88C8
:1039C00004681C4304608B8804681C4304608B6893
:1039D000C36290420FD1136840F20034A3431360D6
:1039E000CB8814681C431460097B01634169012280
:1039F0000A43426110BD124A90420BD0C54A904220
:103A000008D0104A904205D00F4A904202D00F4A87
:103A10009042EBD1026840F200339A430260CA88B8
:103A2000036813430360074A9042DDD0074A90427F
:103A3000DAD0054A9042D7D0D8E7C046002C0140E2
:103A400000040040004001400048014000440140A3
:103A5000C2688A43C2607047C2680A43C260704746
:103A600002698A4302617047C2680A40531E9A4144
:103A700000690840411E88411040704703490022F8
:103A800002730260426081607047C046FFFF000021
:103A9000F0B5FF24094A0A4B25460E0409D00678E2
:103AA0007540565D5F5D25467D40401C491E34468D
:103AB000F3E72002284380B2F0BDC046D04600089C
:103AC000D0450008B0B50D4604467A48844204D07B
:103AD0002048844205D1022000E00520FFF772FE55
:103AE00000E000202168090405D469084018B0FBF3
:103AF000F5F080B209E0690840004018B0FBF5F02D
:103B0000034901400007400F4018E060B0BDC046C7
:103B1000F0FF0000416A034808407047014A0A402C
:103B200082627047FF01000010B56249884204D0EC
:103B3000084988420BD1084C00E0054C2046FFF7AD
:103B4000E9FE204610BC02BC8E46FFF7D9BE10BD70
:103B50000E0300000044004011040000016801222F
:103B60000A43026070471F220A4089090958D14060
:103B70000120084070471F220A4001239340890911
:103B80000A589A430A5070471F220A400123934063
:103B900089090A581A430A5070470000084A91429E
:103BA00006D1D021425848F200039A434250704750
:103BB000C902C90E01228A40016A1143016270479D
:103BC00009340F341F220A400B049B0D1B58D340AD
:103BD0008A0D1258C802C00EC2401A40012010407F
:103BE0007047026801239A430260026840F2006352
:103BF0009A43026002680A43026070470268042325
:103C00009A43026002680A43026070470268012317
:103C10009A430260426843F200039A43426042685A
:103C20000A4342607047026808239A4302600268B0
:103C30000A4302607047026801239A4302600268E7
:103C400041F200039A43026002680A43026070472F
:103C500070B50E460921CC06CB4D0521012808D1AF
:103C60002846FFF791FF204640F60001FFF74DFA86
:103C700007E02846FFF77FFF204640F60001FFF7E8
:103C800046FA06212846012E09D1FFF77DFF20467E
:103C900040F6000170BC04BC9646FFF738BAFFF747
:103CA0006AFF204640F6000170BC04BC9646FFF750
:103CB0002CBAC04600380140B0B5164C0021204651
:103CC000FFF734FE012520462946FFF7C9FE2046AE
:103CD0002946FFF7BDFE2046B0BC02BC8E46FFF76A
:103CE00057BEC04600200040B0B50A4C0021204617
:103CF000FFF71CFE012520462946FFF7B1FE2046AE
:103D00002946FFF7A9FE2046B0BC02BC8E46FFF74D
:103D100044BEC04600200040BCB53A4DA8780028FB
:103D20006AD101A800F028F96878002478B1022847
:103D300018D001285ED1FFF7D7FF01A800780D2821
:103D400028D000243A2828D1EC70AC8052E001A899
:103D500000783A284ED1FFF7C7FF0024AC80EC7002
:103D6000012018E001A800782978884208D1FFF7DF
:103D7000A3FF00206870012000F0F6F8044639E047
:103D800000243A2810D1EC70AC8001206870FFF755
:103D9000ABFF2FE0022068702CE001464139C9B228
:103DA000062903D3E14303E06C7023E00146373971
:103DB0003038C2B20A2A00D30846E97801290AD06D
:103DC000C1B9A988FF2911D8A9880001E54A505432
:103DD0000120E8700EE0A988E24A535C0343535483
:103DE000A888401CA8800024EC7003E000246C70BC
:103DF000FFF762FF2046BCBD03A05149E322FEF756
:103E000045FBC046C401002065536E645374617461
:103E100065203D3D2053544154455F54585F49440B
:103E20004C45000080B53E484178491E012902D822
:103E30000021417005E04178012902D04078022834
:103E400003D1FFF739FF002080BD03483C4940F211
:103E5000A712FEF71BFBC046D847000870B5304ECE
:103E60007078002856D1B078042840D8810001A28B
:103E700051188F4600F008B800F027B800F009B8D4
:103E800000F02BB800F014B801200021FFF7E0FE8D
:103E90002DE0F08830B3F07801282AD038BBB06824
:103EA00000780009FFF76EFC00F0E0F8012012E056
:103EB0000024B470032000F057F805460120214685
:103EC000FFF7C6FEB470284670BD3A2000F0CEF869
:103ED0000220B0700020F07009E0307800F0C6F8E1
:103EE000042003E00D2000F0C1F80320B070002092
:103EF00070BDB06801780F200840FFF743FC00F068
:103F0000B5F80020F070B068401CB060F088401E2A
:103F1000F080ECE703A00A4940F24F12FEF7B6FA30
:103F2000C4010020655263765374617465203D3D81
:103F30002053544154455F52585F49444C4500005A
:103F40001C4800080B490A78012A05D14A780270FA
:103F500000200870012070470020704705480021AC
:103F6000017001207047C046024948700120087066
:103F70007047C046D001002010B504463F48FFF707
:103F8000C9FD2070012010BD00380140FEB502912E
:103F90001B2000252946FFF7ABFB3148FFF7A6FCA5
:103FA0000920C60601243046214640F20022FFF7D0
:103FB00081F8022101913046224640F20023294F28
:103FC000B847294F30462946224640F20023B847D9
:103FD0003046214640F20042FFF76CF83046019926
:103FE000224640F200431F4FB8473046294622463A
:103FF00040F200431C4FB847304621462A4640F65F
:104000000003184FB84703223046294640F6000304
:10401000154EB0471248FD30FFF768FC174E30468A
:10402000FFF782FD30460299FFF74CFD30462946E6
:10403000FFF7ECFD30462946FFF7FDFD30462946E7
:10404000FFF7CFFD04213046FFF7D8FD08213046A9
:10405000FFF7E9FD3046FFF781FD2046FEBDC04673
:1040600011050000213100085F31000880B50146CC
:104070000248FFF753FD012080BDC04600380140D3
:104080007FB5054640F20870FFF730FC104C204623
:10409000FFF74EFC6E463046FFF7F0FC0D483080CF
:1040A000681E02900020019020463146FFF77AFCFE
:1040B000012520462946FFF7CFFC13202946FFF7AC
:1040C00017FB2046FFF769FC284604B070BDC046C8
:1040D000002000400F0E00001CB51A4C607858BB41
:1040E00001A8FFF749FF2078032823D8810001A207
:1040F00051188F4600F01CB800F004B800F00CB85E
:1041000000F016B8002060806088411C618015496D
:10411000019A0A5402200AE06088800A06D1608869
:10412000411C61800F49019A0A5401E0032020706C
:10413000FFF7DAFD00201CBD03A03D49F022FEF789
:10414000A5F9C046F801002065536E64537461748C
:1041500065203D3D2053544154455F54585F4944C8
:104160004C450000BA050020B0B5294D2878002440
:10417000032808D0022802D058B9002000E001200E
:10418000FFF7F2FE0446FFF797FD01202870204656
:10419000B0BD28780028F6D028780228F3D02878F7
:1041A0000328F0D00248224940F26512FEF76EF96A
:1041B0003A48000870B5164E3078012822D1707840
:1041C000012805D080B901200021FFF741FD0BE057
:1041D000B08858B1B0680078FFF748FFB068401C5D
:1041E000B060B088401EB080002070BD0320FFF793
:1041F000BBFE0446012000252946FFF729FD757006
:10420000204670BD03A00A4940F22B12FEF73EF98A
:10421000F8010020655263765374617465203D3D5A
:104220002053544154455F52585F49444C45000067
:104230009D48000810B500F01FF8EFF300808000E3
:1042400001D4012010BD002010BD10B500F08CF885
:10425000EFF30080800001D5012010BD002010BDCB
:1042600010B500F0ABF8EFF30080800001D401201E
:1042700010BD002010BD000070B501252D050C00FB
:104280001C4310D4EC4206D4AC420AD4994200D06C
:1042900070BD904270BDE94217D4EB4215D49942EB
:1042A00070BD894270BDEC4206D5AC42F9D58B4257
:1042B00000D070BD824270BD6D004C00EC4204D253
:1042C0005C00EC4201D28B4270BD034C30B4FCF771
:1042D0004FFA30BC70BD00BF1900160470B501253F
:1042E000ED0704004C4020D4441A01D2001B0919E8
:1042F000C60D4B00F2B2FF2A29D01B0E2CD00002B3
:104300000C0228432C43D31ADC40051910D2280A8A
:1043100002D3401C6D0611D0761EF6058019FF2AC7
:1043200000DA70BDC00DC00570BD694000F0CEF868
:1043300001200543C541521C761CE8E764089C40F7
:10434000C90161408900E7D10124A043E4E71B0EC5
:10435000440200D0034870BD002AFCD1C00FC00742
:1043600070BD00BF0000C07F0123DB0502000A43CF
:104370000DD4DA4203D49A4207D488427047D84217
:1043800014D4D94212D48842704780427047DA422E
:1043900003D59A42F9D5814270475B004200DA4268
:1043A00004D24A00DA4201D28142704710B5024A73
:1043B000FCF72EFA10BD00BF090013040123DB0532
:1043C00002000A430DD4DA4203D49A4207D4884249
:1043D0007047D84214D4D94212D4884270478042E0
:1043E0007047DA4203D59A42F9D5814270475B00A3
:1043F0004200DA4204D24A00DA4201D281427047D6
:1044000010B5024AFCF704FA10BD00BF09001604FB
:1044100070B5420064414B005C41120E39D01B0E56
:1044200038D0FF2A3CD0FF2B3AD0D2187F3A400236
:104430004902400A490A4518ED0106004E43000AA8
:10444000090A48430104731A4019190C4318990FBB
:1044500004D05B08012149075B1A521CD80904D318
:10446000401CF50301D19D0607D0FF2A08D2D505CF
:1044700006D0E4072043401970BD0125A843F4E7A6
:10448000002A01DCE00770BD2402FF202043C005A4
:1044900070BD1B0EFF2A03D0FF2B01D0E00770BDBB
:1044A000FF2636064500B54206D84D00B54203D872
:1044B000D218FF2A00D0E7E7004870BD0000C07F97
:1044C00070B50125ED0704004C4022D4441A02D2F5
:1044D0006C40001B0919C60D4B00F2B2FF2A4BD0ED
:1044E0001B0E50D000020C02A8432C43D31ADC4010
:1044F000051B05D5AD0019D36D08761E521E37D0A9
:10450000F605280A01D2801970BD70416D0603D0EE
:1045100070BD6940FFF7E8FE9C4009026140490018
:1045200001D0401E70BD0124A04370BD6D081DD098
:1045300001202B0C01D12D0410302B0E01D12D02A6
:1045400008302B0F01D12D01001DAB0F01D1AD00A3
:10455000801CEB0F01D16D00401C361A121A6D0041
:10456000680AF5054019012A02DB70BD002070BD04
:10457000C036300AC00770BD1B0E440201D1FF2BAC
:1045800000D1024870BD002AF0D070BD0000C07F8D
:104590008182838485868788898B8C8D8E8F91928A
:1045A00093959697999A9C9D9FA0A2A3A5A7A8AA28
:1045B000ACAEB0B2B3B5B7B9BCBEC0C2C5C7C9CC4A
:1045C000CED1D4D7D9DCDFE2E6E9ECF0F3F7FAFE9E
:1045D00000C1814001C0804101C0804100C18140D3
:1045E00001C0804100C1814000C1814001C08041C3
:1045F00001C0804100C1814000C1814001C08041B3
:1046000000C1814001C0804101C0804100C18140A2
:1046100001C0804100C1814000C1814001C0804192
:1046200000C1814001C0804101C0804100C1814082
:1046300000C1814001C0804101C0804100C1814072
:1046400001C0804100C1814000C1814001C0804162
:1046500001C0804100C1814000C1814001C0804152
:1046600000C1814001C0804101C0804100C1814042
:1046700000C1814001C0804101C0804100C1814032
:1046800001C0804100C1814000C1814001C0804122
:1046900000C1814001C0804101C0804100C1814012
:1046A00001C0804100C1814000C1814001C0804102
:1046B00001C0804100C1814000C1814001C08041F2
:1046C00000C1814001C0804101C0804100C18140E2
:1046D00000C0C101C30302C2C60607C705C5C404A2
:1046E000CC0C0DCD0FCFCE0E0ACACB0BC90908C812
:1046F000D81819D91BDBDA1A1EDEDF1FDD1D1CDC02
:1047000014D4D515D71716D6D21213D311D1D01071
:10471000F03031F133F3F23236F6F737F53534F461
:104720003CFCFD3DFF3F3EFEFA3A3BFB39F9F838D1
:1047300028E8E929EB2B2AEAEE2E2FEF2DEDEC2CC1
:10474000E42425E527E7E62622E2E323E12120E031
:10475000A06061A163A3A26266A6A767A56564A421
:104760006CACAD6DAF6F6EAEAA6A6BAB69A9A86891
:1047700078B8B979BB7B7ABABE7E7FBF7DBDBC7C81
:10478000B47475B577B7B67672B2B373B17170B0F1
:1047900050909151935352929656579755959454E1
:1047A0009C5C5D9D5F9F9E5E5A9A9B5B9959589851
:1047B000884849894B8B8A4A4E8E8F4F8D4D4C8C41
:1047C00044848545874746868242438341818040B1
:1047D0000000000001020304282065526376537430
:1047E000617465203D3D2053544154455F52585FEC
:1047F0005243562029207C7C202820655263765322
:1048000074617465203D3D2053544154455F5258B6
:104810005F574149545F454F462029002E2E2F41B6
:1048200070702F4D6F646275732F61736369692FA8
:104830006D6261736369692E630028206552637637
:104840005374617465203D3D2053544154455F527B
:10485000585F494E49542029207C7C2028206552ED
:1048600063765374617465203D3D20535441544533
:104870005F52585F5243562029207C7C20282065B7
:104880005263765374617465203D3D205354415406
:10489000455F52585F4552524F522029002E2E2F0D
:1048A0004170702F4D6F646275732F7274752F6D28
:1048B000627274752E630000D84800080000002062
:1048C00090000000100100086849000890000020D6
:1048D000001900002C010008060100001E00000065
:1048E00000A24A040200000011000000092800088C
:1048F000040000000927000803000000B12600089A
:1049000010000000F9280008060000006D280008CB
:10491000170000006B27000801000000CD250008EB
:1049200005000000292800080F0000009F2800084B
:10493000020000003D26000800000000000000000A
:104940000000000000000000000000000000000067
:104950000000000000000000000000000000000057
:0849600000000000000000004F
:04000005080000CD22
:00000001FF
